:1000000012C0189518951895189518951895189563
:100010008CC6D2C2189518951895189518951895EC
:100020001895189518958FE58DBFC8E3E0E24E2E20
:1000300084E08EBFD4E0F4E05F2EA89584B7082E4C
:10004000877F84BF88E1992781BD91BDEEEFF3E002
:10005000A0E6B0E088278D933197E9F76624A09851
:10006000A89AA198A99AA298AA9A8FEF81BB8FEF1C
:1000700087BB86E886B980E487B981E08093620017
:1000800000916200063010F009F015C08BE090E09E
:10009000A2E6B0E0AD90BB24A3E6B0E0AA0CBB1C86
:1000A000AA0DBB1D8D939C93A2E6B0E08C918F5F4F
:1000B0008C9308F4E5CFEAE1F0E0A2E9B0E091E04A
:1000C00097DC989957C081E08093620000916200AC
:1000D000083C10F009F04EC000916200063909F0AA
:1000E0003CC080918C00806880938C00A2E9B0E0D5
:1000F0008C9198E089278C93EAE1F0E0A2E9B0E0E6
:1001000091E07BE764DC00919200003009F00EC0C2
:1001100092989698C798C2989098C6989798C598BC
:10012000939A949A919A959AC09AC19A0091920042
:10013000083009F00EC0929A969AC79AC29A909A7D
:10014000C69A979AC59A9398949891989598C098BA
:10015000C1988CED95E054DA0DC0989B01C00AC09F
:100160008AE090E04DDAA2E6B0E08C918F5F8C934C
:1001700008F4ACCFE4E1F0E0A0E1B0E036DC0F3F02
:1001800009F05AC088E290E0A5E7B0E08D939C9317
:1001900084E190E0A3E7B0E08D939C9380E293E04C
:1001A000ABE7B0E08D939C9384E893E0A9E7B0E0DF
:1001B0008D939C9388E0809392008BEB80938F00CB
:1001C0008BEB80939000E0E0F0E0A3E7B0E092E0FA
:1001D0007BE7FDDBE5E0F0E0A5E7B0E092E07BE760
:1001E000F6DBEAE0F0E0A9E7B0E092E07BE7EFDBE6
:1001F000EEE0F0E0ABE7B0E092E07BE7E8DBE0E1E7
:10020000F0E0AFE8B0E091E07BE7E1DBE1E1F0E0D6
:10021000A0E9B0E091E07BE7DADBEAE1F0E0A2E917
:10022000B0E091E07BE7D3DBE4E1F0E0A0E1BB27C5
:1002300084E68C937BE7C8DBE0E0F0E0A3E7B0E086
:1002400092E0D6DBE5E0F0E0A5E7B0E092E0D0DBBD
:10025000EAE0F0E0A9E7B0E092E0CADBEEE0F0E02F
:10026000ABE7B0E092E0C4DBE0E1F0E0AFE8B0E0A3
:1002700091E0BEDBE1E1F0E0A0E9B0E091E0B8DBC5
:1002800083E083BF80E08FBD81E08EBD789489B725
:10029000816089BF89B7846089BF83E083BF81E0C3
:1002A0008EBD379A82E3809362000091620008322B
:1002B00010F009F001C023C0882783BF8EB5887F66
:1002C0008EBD80918C00826080938C0080E0809352
:1002D000620007B1007F056007B9A1D9A8E9B0E0C5
:1002E0008D939C9307B1007F046007B998D9AAE960
:1002F000B0E08D939C9383E083BF81E08EBD8091BD
:100300008C008D7F80938C00E4E3FBE139DBE8E92E
:10031000F0E0D190E0808FEFE7FE8827F82E082FDD
:10032000F3D943DAEDE0F0E0A4E9B0E041DBE4E941
:10033000F0E0CBD9E8E3FBE11ADB8DDAEDE0F0E0A9
:10034000A4E9B0E035DBE4E9F0E08BDBEDE0F0E0E0
:10035000A4E9B0E02DDB0FEF13E0A8E9B0E04D9188
:100360005C91041B150BA8E9B0E00D931C93A8E960
:10037000B0E00D911C914CE050E0FFD8A8E9B0E04E
:100380004D935C93E4E9F0E0A0D9E8E9F0E0D19086
:10039000E0808FEFE7FE8827F82E082FB5D95BDACB
:1003A000EDE0F0E0A4E9B0E003DBE4E9F0E04AD9F5
:1003B000A8E9B0E0EE0C000FE794DD92EC92A8E91A
:1003C000B0E00D911C91053550E0150714F009F0CF
:1003D00001C006C085E590E0A8E9B0E08D939C934C
:1003E0000FEF13E0AAE9B0E04D915C91041B150BEF
:1003F000AAE9B0E00D931C93AAE9B0E00D911C911D
:1004000041E050E0BAD8AAE9B0E04D935C93AAE984
:10041000B0E00D911C91073E53E0150714F009F070
:1004200001C006C087EE93E0AAE9B0E08D939C93EB
:10043000882783BF8EB5887F8EBDA8E9B0E08D91F7
:100440009C91A1E7B0E08D939C93AAE9B0E08D91D7
:100450009C91A7E7B0E08D939C9383E083BF81E0FC
:100460008EBDA5E7B0E04D915C91A3E7B0E00D91A2
:100470001C910417150708F021C0A3E7B0E04D91C7
:100480005C91A1E7B0E00D911C910417150714F0E1
:1004900009F003C081E080937D00A5E7B0E04D91B5
:1004A0005C91A1E7B0E00D911C91041715070CF0C9
:1004B00001C003C080E080937D0020C0A3E7B0E0CE
:1004C0004D915C91A1E7B0E00D911C9104171507C7
:1004D0000CF001C003C081E080937D00A5E7B0E08F
:1004E0004D915C91A1E7B0E00D911C9104171507A7
:1004F00014F009F003C080E080937D0000917D003E
:10050000013009F002C0C39A01C0C398ABE7B0E064
:100510004D915C91A9E7B0E00D911C91041715076E
:1005200008F021C0A9E7B0E04D915C91A7E7B0E0E9
:100530000D911C910417150714F009F003C081E018
:1005400080937E00ABE7B0E04D915C91A7E7B0E00F
:100550000D911C91041715070CF001C003C080E039
:1005600080937E0020C0A9E7B0E04D915C91A7E7A1
:10057000B0E00D911C91041715070CF001C003C0E9
:1005800081E080937E00ABE7B0E04D915C91A7E7FE
:10059000B0E00D911C910417150714F009F003C089
:1005A00080E080937E0000917E00013009F002C05F
:1005B000C49A01C0C49879CE0F921F922F923F9295
:1005C0004F925F927F92AF92BF920F931F932F93A0
:1005D0003F934F935F936F937F938F939F93AF93CB
:1005E000BF93CF93DF93EF93FF938FB78F930091D8
:1005F0008B00003081E009F480E08F93ACE8B0E03C
:100600008C9185FB81E00EF480E09F918923882303
:1006100009F403C0ADE8B0E09FD7ADE8B0E00D91BC
:100620001C9108355BE1150710F009F001C009C005
:1006300080E090E0ADE8B0E08D939C9380E0809303
:100640008B00882783BF00918B00003009F011C018
:10065000A1E7B0E08D919C91A5E8B0E08D939C93CB
:10066000A7E7B0E08D919C91A7E8B0E08D939C93B3
:100670004FC0013009F011C0A3E7B0E08D919C910B
:10068000A5E8B0E08D939C93A7E7B0E08D919C9195
:10069000A7E8B0E08D939C933BC0023009F011C0F5
:1006A000A5E7B0E08D919C91A5E8B0E08D939C9377
:1006B000A7E7B0E08D919C91A7E8B0E08D939C9363
:1006C00027C0033009F011C0A1E7B0E08D919C91E3
:1006D000A5E8B0E08D939C93A9E7B0E08D919C9143
:1006E000A7E8B0E08D939C9313C0043009F010C0CC
:1006F000A1E7B0E08D919C91A5E8B0E08D939C932B
:10070000ABE7B0E08D919C91A7E8B0E08D939C930E
:10071000ACE8B0E08C9183FB0EF44FC0A5E8B0E0EC
:100720008D919C91AFE7B0E08D939C93AFE7B0E0E3
:100730008D919C91A3E8B0E08D939C9383E080938E
:1007400063004091630001E0041710F009F025C038
:10075000AFE7B0E00D911C914AE050E00ED7A3E660
:10076000B0E0AD90BB24A3E6B0E0AA0CBB1CAA0D80
:10077000BB1D0D931C93AFE7B0E00D911C914AE0B7
:1007800050E0FBD6AFE7B0E04D935C9380916300FF
:1007900081508093630008F0D4CFA3E8B0E00D91BE
:1007A0001C91043650E015070CF401C006C08BE024
:1007B00090E0A5E6B0E08D939C93ACE8B0E08C911E
:1007C00082FB0EF44FC0A7E8B0E08D919C91A1E8A8
:1007D000B0E08D939C93A1E8B0E08D919C91A3E84B
:1007E000B0E08D939C9386E080936300409163001A
:1007F00004E0041710F009F025C0A1E8B0E00D9165
:100800001C914AE050E0B9D6A3E6B0E0AD90BB241D
:10081000A3E6B0E0AA0CBB1CAA0DBB1D0D931C9354
:10082000A1E8B0E00D911C914AE050E0A6D6A1E805
:10083000B0E04D935C93809163008150809363009E
:1008400008F0D4CFA3E8B0E00D911C91043650E03D
:1008500015070CF401C006C08BE090E0ABE6B0E0F9
:100860008D939C9300919200003009F007C09398FB
:10087000949891989598C098C19806C0939A949A24
:10088000919A959AC09AC19AA0E6B0E08C918F5F38
:100890008C9300916000063010F009F001C003C095
:1008A00081E08093600080E08093610090D1A4E6B5
:1008B000B0E08C9180FBA2E3B0E08C9182F98C9344
:1008C00086D1A4E6B0E08C9180FBA2E3B0E08C91ED
:1008D00086F98C937CD1A4E6B0E08C9180FBA8E3F0
:1008E000B0E08C9187F98C9372D1A4E6B0E08C9142
:1008F00080FBA8E3B0E08C9182F98C9368D1A4E6E8
:10090000B0E08C9180FBA2E3B0E08C9180F98C93F5
:100910005ED1A4E6B0E08C9180FBA8E3B0E08C91BE
:1009200086F98C9354D1A4E6B0E08C9180FBA2E3CD
:10093000B0E08C9187F98C9300916000013009F050
:100940002FC000919200003009F013C0919AACE8DA
:10095000B0E08C9183FB0EF40AC0AFE8B0E08C915C
:1009600083FBA8E3B0E08C9185F98C9301C0C59A14
:1009700016C09198ACE8B0E08C9183FB0EF40EC0E9
:10098000AFE8B0E08C9183FBA8E3B0E08C9185F9EF
:100990008C9388B390E2892788BB01C0C598F9C0C1
:1009A000023009F02FC000919200003009F013C00E
:1009B000949AACE8B0E08C9183FB0EF40AC0AFE8E7
:1009C000B0E08C9182FBA8E3B0E08C9185F98C9328
:1009D00001C0C59A16C09498ACE8B0E08C9183FB36
:1009E0000EF40EC0AFE8B0E08C9182FBA8E3B0E05B
:1009F0008C9185F98C9388B390E2892788BB01C0DC
:100A0000C598C7C0033009F02FC000919200003094
:100A100009F013C0939AACE8B0E08C9183FB0EF41C
:100A20000AC0AFE8B0E08C9181FBA8E3B0E08C9104
:100A300085F98C9301C0C59A16C09398ACE8B0E0D4
:100A40008C9183FB0EF40EC0AFE8B0E08C9181FB7B
:100A5000A8E3B0E08C9185F98C9388B390E2892764
:100A600088BB01C0C59895C0043009F02FC0009123
:100A70009200003009F013C0C19AACE8B0E08C914C
:100A800082FB0EF40AC0A0E9B0E08C9183FBA8E3DE
:100A9000B0E08C9185F98C9301C0C59A16C0C198BD
:100AA000ACE8B0E08C9182FB0EF40EC0A0E9B0E09F
:100AB0008C9183FBA8E3B0E08C9185F98C9388B38B
:100AC00090E2892788BB01C0C59863C0053009F052
:100AD0002FC000919200003009F013C0C09AACE81A
:100AE000B0E08C9182FB0EF40AC0A0E9B0E08C91DA
:100AF00082FBA8E3B0E08C9185F98C9301C0C59A84
:100B000016C0C098ACE8B0E08C9182FB0EF40EC029
:100B1000A0E9B0E08C9182FBA8E3B0E08C9185F96C
:100B20008C9388B390E2892788BB01C0C59831C0F7
:100B3000063009F02EC000919200003009F013C079
:100B4000959AACE8B0E08C9182FB0EF40AC0A0E963
:100B5000B0E08C9181FBA8E3B0E08C9185F98C9397
:100B600001C0C59A16C09598ACE8B0E08C9182FBA4
:100B70000EF40EC0A0E9B0E08C9181FBA8E3B0E0D8
:100B80008C9185F98C9388B390E2892788BB01C04A
:100B9000C59883E083BF8F918FBFFF91EF91DF9165
:100BA000CF91BF91AF919F918F917F916F915F9105
:100BB0004F913F912F911F910F91BF90AF907F90D8
:100BC0005F904F903F902F901F900F901895A0E648
:100BD000B0E0AD90BB24A3E6B0E0AA0CBB1CAA0D0C
:100BE000BB1D0C9147E0049FA4E6B0E00C9200917D
:100BF000610040916400040FA4E6B0E00C93009102
:100C00009200003009F00AC0EAE3FCE0A4E6B0E09C
:100C10008C919927A4E6B0E0C8D609C0E2EBFCE0CD
:100C2000A4E6B0E08C919927A4E6B0E0BED6A1E698
:100C3000B0E08C918F5F8C9308950000000000005D
:100C4000010100000101010100000100000100009C
:100C5000000000010100010000010100000001008E
:100C60000001000000010000000000000000010180
:100C70000101000000000000000000000001000071
:100C80000101010101010001010101010101010155
:100C9000010000000101010001000100000101014B
:100CA000000000000101000000000101010100013D
:100CB000000001010101010100000101000000002C
:100CC0000101000101000101010101000001000119
:100CD0000100000101010001010001010100010109
:100CE00001010101010100000000010101010101F8
:100CF00001010101010001010000000000000100EC
:100D000000000000000000000001010100000001DF
:100D100000010001010000000101010100000101CA
:100D2000010100000000010001000F921F922F92AC
:100D30003F924F925F927F92AF92BF920F931F9319
:100D40002F933F934F935F936F937F938F939F93D3
:100D5000AF93BF93CF93DF93EF93FF938FB78F93AF
:100D6000A2E6B0E08C918F5F8C938EB5887F8EBDAC
:100D7000A3E3B0E00C9100FB81E00EF480E08F93E0
:100D8000ACE8B0E08C9187FB81E00EF480E09F91AD
:100D900089238F93A3E3B0E00C9101FB81E00EF077
:100DA00080E09F9189238F93A3E3B0E00C9102FB35
:100DB00081E00EF080E09F918923882309F401C02F
:100DC000B4D0ACE8B0E08C9184FB81E00EF080E020
:100DD0008F93A3E3B0E00C9100FB81E00EF080E084
:100DE0009F918923882309F406C0999901C0DED216
:100DF0009A9901C02CD3A3E3B0E00C9100FB81E0F1
:100E00000EF480E08F93A3E3B0E00C9101FB81E04E
:100E10000EF480E09F9189238F9300918B00003026
:100E200081E009F080E09F9189238F93ACE8B0E0E6
:100E30008C9186FB81E00EF480E09F9189238823CA
:100E400009F401C05DD3A3E3B0E00C9100FB81E0A5
:100E50000EF480E08F93A3E3B0E00C9102FB81E0FD
:100E60000EF480E09F9189238F9300918B000030D6
:100E700081E009F080E09F9189238F93ACE8B0E096
:100E80008C9186FB81E00EF480E09F91892388237A
:100E900009F401C04BD3A3E3B0E00C9100FB81E067
:100EA0000EF080E08F93A3E3B0E00C9101FB81E0B2
:100EB0000EF080E09F9189238F93A3E3B0E00C9123
:100EC00002FB81E00EF080E09F918923882309F4E2
:100ED00005C080918C008F7780938C00989B05C013
:100EE00080918C008F7B80938C0081E08EBD83E0AD
:100EF00083BF8F918FBFFF91EF91DF91CF91BF9112
:100F0000AF919F918F917F916F915F914F913F91A1
:100F10002F911F910F91BF90AF907F905F904F9056
:100F20003F902F901F900F901895789489B781600B
:100F300089BF83E083BF80918C00806180938C00A7
:100F400080918C00806880938C0080E090E0ADE818
:100F5000B0E08D939C93A5E7B0E04D915C91A3E741
:100F6000B0E00D911C910417150781E009F080E0B5
:100F70008F93ABE7B0E04D915C91A9E7B0E00D91A4
:100F80001C910417150781E009F080E09F91892BDF
:100F9000882309F401C0FDD0ABE8B0E08C918F5FED
:100FA0008C9300918B00043010F009F001C003C055
:100FB00080E080938B0000918B00003009F043C0EB
:100FC00080918C00886080938C0080918C0084607C
:100FD00080938C008AE090E0A5E6B0E08D939C932E
:100FE0008AE090E0A7E6B0E08D939C938AE090E0E1
:100FF000A9E6B0E08D939C938AE090E0ABE6B0E088
:101000008D939C938AE090E0ADE6B0E08D939C9345
:101010008AE090E0AFE6B0E08D939C9380918C00E5
:101020008F7E80938C0084EF91E0EAD28EB5887F2A
:101030008EBD882783BFEEE0F0E0ABE7B0E092E042
:101040007BE7C5D49BC0013009F01BC080918C00A8
:10105000886080938C0081E090E0A9E6B0E08D93F9
:101060009C938DE090E0A7E6B0E08D939C9380E0A8
:1010700090E0A5E6B0E08D939C9384EF91E0C0D220
:101080007DC0023009F027C080918C008860809379
:101090008C0081E090E0A9E6B0E08D939C938EE017
:1010A00090E0A7E6B0E08D939C9380E090E0A5E609
:1010B000B0E08D939C9384EF91E0A2D28EB5887FAF
:1010C0008EBD882783BFE0E0F0E0A3E7B0E092E0C8
:1010D0007BE77DD453C0033009F027C080918C009A
:1010E000846080938C0082E090E0AFE6B0E08D9366
:1010F0009C938DE090E0ADE6B0E08D939C9380E012
:1011000090E0ABE6B0E08D939C9384EF91E078D2D1
:101110008EB5887F8EBD882783BFE5E0F0E0A5E728
:10112000B0E092E07BE753D429C0043009F026C038
:1011300080918C00846080938C0082E090E0AFE628
:10114000B0E08D939C938EE090E0ADE6B0E08D939F
:101150009C9380E090E0ABE6B0E08D939C9384EFAD
:1011600091E04ED28EB5887F8EBD882783BFEAE09E
:10117000F0E0A9E7B0E092E07BE729D480918C0011
:10118000877F80938C0080918C008B7F80938C0074
:10119000089580918C00806280938C00A5E7B0E078
:1011A0004D915C91A3E7B0E00D911C9104171507D8
:1011B00009F059C080918C00886080938C008FE08A
:1011C00090E0A5E6B0E08D939C9380E190E0A7E6E7
:1011D000B0E08D939C9380E190E0A9E6B0E08D9320
:1011E0009C9384EF91E00CD28BE090E0A5E6B0E018
:1011F0008D939C938BE090E0A7E6B0E08D939C9359
:101200008BE090E0A9E6B0E08D939C9384EF91E0B1
:10121000F7D18FE090E0A5E6B0E08D939C9380E15C
:1012200090E0A7E6B0E08D939C9380E190E0A9E682
:10123000B0E08D939C9384EF91E0E2D18BE090E05D
:10124000A5E6B0E08D939C938BE090E0A7E6B0E03C
:101250008D939C938BE090E0A9E6B0E08D939C93F6
:1012600084EF91E0CDD1ABE7B0E04D915C91A9E77F
:10127000B0E00D911C910417150709F059C0809139
:101280008C00846080938C008FE090E0ABE6B0E04F
:101290008D939C9380E190E0ADE6B0E08D939C93BC
:1012A00080E190E0AFE6B0E08D939C9384EF91E015
:1012B000A7D18BE090E0ABE6B0E08D939C938BE000
:1012C00090E0ADE6B0E08D939C938BE090E0AFE6CC
:1012D000B0E08D939C9384EF91E092D18FE090E009
:1012E000ABE6B0E08D939C9380E190E0ADE6B0E09A
:1012F0008D939C9380E190E0AFE6B0E08D939C935A
:1013000084EF91E07DD18BE090E0ABE6B0E08D938F
:101310009C938BE090E0ADE6B0E08D939C938BE0E6
:1013200090E0AFE6B0E08D939C9384EF91E068D1BC
:1013300000918B00003009F001C027C0013009F096
:1013400007C0E0E0F0E0A3E7B0E092E051D31DC0B9
:10135000023009F007C0E5E0F0E0A5E7B0E092E078
:1013600047D313C0033009F007C0EAE0F0E0A9E773
:10137000B0E092E03DD309C0043009F006C0EEE0D1
:10138000F0E0ABE7B0E092E033D380918B00815086
:1013900080938B0080E090E0ADE8B0E08D939C936B
:1013A00080918C008F7D80938C000895789489B70C
:1013B000816089BF83E083BF80E090E0ADE8B0E06A
:1013C0008D939C9300918B00013009F00DC0A3E731
:1013D000B0E00D911C91053550E0150708F003C0F1
:1013E000A3E7B0E0B9D02FC0023009F00DC0A5E7E7
:1013F000B0E00D911C91053550E0150708F003C0D1
:10140000A5E7B0E0A9D01FC0033009F00DC0A9E7DF
:10141000B0E00D911C91053550E0150708F003C0B0
:10142000A9E7B0E099D00FC0043009F00CC0ABE7D9
:10143000B0E00D911C91053550E0150708F003C090
:10144000ABE7B0E089D08FE090E0DAD008957894EF
:1014500089B7816089BF83E083BF80E090E0ADE819
:10146000B0E08D939C9300918B00013009F00FC088
:10147000A3E7B0E00D911C91003050E0150710F08B
:1014800009F001C003C0A3E7B0E06DD035C0023061
:1014900009F00FC0A5E7B0E00D911C91003050E0BD
:1014A000150710F009F001C003C0A5E7B0E05BD05C
:1014B00023C0033009F00FC0A3E7B0E00D911C91E9
:1014C000003050E0150710F009F001C003C0A9E793
:1014D000B0E049D011C0043009F00EC0ABE7B0E075
:1014E0000D911C91003050E0150710F009F001C07B
:1014F00003C0ABE7B0E037D08FE090E081D0089533
:1015000080918C00806480938C0091E0AFE8B0E023
:101510008FD08EB5887F8EBD882783BFE0E1F0E055
:10152000AFE8B0E091E07BE752D2089580918C0063
:10153000806480938C0091E0A0E9B0E079D08EB512
:10154000887F8EBD882783BFE1E1F0E0A0E9B0E0AD
:1015500091E07BE73CD20895ED91FC91EF5FFF4F66
:10156000FC93EE930895ED91FC91E150F040FC93D3
:10157000EE93089500FC10D0089503D01ED001F81A
:10158000F9CF0024E89457FF02C009D0689400F80E
:101590000BD010F80124089502D009D00895509579
:1015A00040954F5F5F4F0895E89417FF08950095A9
:1015B00010950F5F1F4F68940895352F242FE894DE
:1015C000452B11F468940895512F402F00271127BF
:1015D00080E1440F551F001F111F021B130B4160B8
:1015E00018F4020F131F4E7F8A9599F708953197CB
:1015F000F1F70895689462F80895E89462F8089500
:10160000EF93FF93EE27E82BE92B31F0E0EDF7E0C5
:101610003197F1F70197D1F7FF91EF910895369A3D
:101620003699FECF369A3699FECF84B195B108959A
:10163000903039F08C91880F08F481609A95D9F731
:101640008C9308953DD0992711278F2D880F80E81E
:10165000F82A802F881F08F41FEF41F08F57082FBA
:1016600007FD04C0003240F08FEF01C08827982F9B
:10167000D82EE82EF82E09C08FE1801B082FF69493
:10168000E794D79497950A95D1F7112351F0909547
:10169000D094E094F09481E0980F8827D81EE81E3B
:1016A000F81E0F2DFE2CED2CD92E0895D094E09429
:1016B000F09491E0D90E9927E91EF91E109508952E
:1016C000D190E190F1900191089521913191419152
:1016D00051910895102F90E8FF0C001F0927990FD2
:1016E000F7941078652F90E8440F551F5927990FEC
:1016F0004795607800380895FF0C90E89027110F07
:101700009795F794092F0895102FBD2CDE2CEF2C00
:10171000F02E11234AF4B094D094E094F0949FEF0B
:10172000B91AD90AE90AF90A0EE1FF2039F4FE2CA8
:10173000ED2CDB2CBB240850C2F76BC032F00A95AD
:10174000BB0CDD1CEE1CFF1CF9CF01D0D5CFB7FEC2
:10175000089590E8B91611F4D0FE08959FEFD91AB4
:10176000E90AF90A09F403950895DD92ED92FD92D4
:101770000C930895502F2D2D3E2D4F2D612F089540
:101780002DEC3CEC4CEC5DE366270FC099DFF2DFFB
:10179000DD24EE2490E8F92E0FE307C096DF05C0A4
:1017A0002227332740E251E46627552351F10023D5
:1017B00081F190DF71F11627005850580894050BFD
:1017C00018F407FD03C025C007FD23C046953795D3
:1017D0002795F694E794D79422D0FF202AF0DD0CC9
:1017E000EE1CFF1C015073F09D2D969548F0DD20F6
:1017F0003AF4EE202AF491E0D90E9927E91EF91E59
:101800007BCF07C09FE7092FF92A9FEFD92EE92E3A
:101810000895DD24EE24FF240027112708959F92C8
:101820009924AA24BB2488E1D216E306F40628F002
:10183000D21AE30AF40A089401C08894991CAA1CDD
:10184000BB1CDD0CEE1CFF1C8A9571F7D92CEA2C11
:10185000FB2C9F9008953EDFE1F25038D1F216271D
:10186000005850580894051F12F418F4CBCF08F014
:10187000D0CF0BD0FF202AF0BB0CDD1CEE1CFF1CD0
:101880003BCF0F5F0BF4BECF37CF9F929924AA2492
:10189000BB24992788E1990CAA1CBB1CDD1CEE1CFB
:1018A000FF1C30F4920EA31EB41ED91EE91EF91EB1
:1018B0008A9589F79F9008950AF045D01DCF5FE380
:1018C00022273327442701C000DF04DF5038B1F35B
:1018D000003899F3902F951B8BF312F434D0FACF84
:1018E000983118F0222733274427983028F0232FE7
:1018F000342F44279850F9CF992329F046953795EE
:1019000027959A95D9F7912F962742F014D0B0F6E3
:10191000F794E794D7940F5F8BF674CF10D051F003
:1019200008F4C4DEFF2052F2DD0CEE1CFF1C015057
:10193000CBF768CF6ECFD20EE31EF41E0895D21AF5
:10194000E30AF40A0895DF92EF92FF920F931F9338
:10195000D22EE32EF42E052F162F6F915F914F910B
:101960003F912F910895C895319600200895FBDF8F
:10197000D02CF9DFE02CF7DFF02CF5DF002D0895F7
:10198000F2DF202DF0DF302DEEDF402DECDF502D8B
:10199000089591E005C092E003C094E001C098E092
:1019A000E2DF0D929A95E1F70895E80FF91FF1CF64
:1019B00094E081918D939A95E1F70895E199FECF96
:1019C000EEBBFFBB3196089591E001C092E07B37FA
:1019D00051F47FB7F894F2DF8D918DBBE29AE19AD2
:1019E0009A95C9F77FBF7727089591E001C092E0EB
:1019F000E5DFE09A8DB38D939A95D1F7089588E04D
:101A00000FB6F8945A924A92E42DF52DA42DB52DD7
:101A1000480E8827581E0FBE08950FB6F8944990B7
:101A200059900FBE08954CDE55DE0395AAF087E16C
:101A3000DD0CEE1CFF1C8A9589F00A95CAF7FF2081
:101A40005AF000240D280E280F28002039F00A959E
:101A5000DD0CEE1CFF1CDAF70A954ECEDACED2DE94
:101A6000DCCF2EDE86E0CCDF05830F772BE33AEA6E
:101A700048EB5FE3F0DE79DE139741D028F48581EF
:101A800088236AF7C6DEC9CF8F77848319DE34973F
:101A9000CBDF6BDE139723E632E446E357EBDBDE66
:101AA00029ED37EA4AE159E33CD026E538E14EEA30
:101AB0005AEB37D026E53CE84DE15CE332D02DEC23
:101AC00037E543E65DEB2DD02DEE3DEF45E75EE3D8
:101AD00028D028E132E741E35FEB23D026D0F5DEC2
:101AE00049DEDD24EE24FF2404818FE7080F0695EC
:101AF000F7945BDE8581881F08F449DE8ECFEADD2E
:101B00008827039512F48894089507301AF0812FDE
:101B100008940895FF1C881F0A95E2F7812B88948A
:101B20000895D3DED2DD349796CE5FE340E83327C5
:0C1B3000222708950000FA44000080BF46
:00000001FF
